:020000020000FC
:10040000271024722346228F22042190212C20D2EF
:10041000208120371FF21FB11F741F3A1F031ECE09
:100420001E9B1E6B1E3C1E0E1DE21DB81D8E1D6602
:100430001D3E1D181CF21CCE1CAA1C861C641C42EE
:100440001C211C001BE01BC01BA11B821B641B4644
:100450001B281B0B1AEE1AD21AB61A9A1A7E1A63A6
:100460001A481A2E1A1319F919DF19C619AC19935B
:10047000197A1961194919301918190018E818D191
:1004800018B918A2188A1873185C1846182F18186B
:10049000180217EB17D517BF17A91793177E176800
:1004A0001752173D1727171216FD16E816D216BD5C
:1004B00016A91694167F166A16551641162C16188C
:1004C000160315EF15DB15C615B2159E158A1576A0
:1004D0001562154E153A1526151214FE14EA14D697
:1004E00014C214AE149B148714731460144C143883
:1004F0001424141113FD13EA13D613C213AF139B64
:10050000138813741360134D13391325131212FE3D
:1005100012EB12D712C312AF129C1288127412611E
:10052000124D12391225121111FD11E911D511C107
:1005300011AD119911851171115D114911341120FD
:10054000110C10F710E310CE10BA10A51090107B0C
:1005500010661052103D102710120FFD0FE80FD239
:100560000FBD0FA70F910F7C0F660F500F3A0F248E
:100570000F0D0EF70EE00EC90EB30E9C0E850E6D1C
:100580000E560E3E0E270E0F0DF70DDF0DC60DAEEB
:100590000D950D7C0D630D490D300D160CFC0CE115
:1005A0000CC70CAC0C910C750C590C3D0C210C04B7
:1005B0000BE70BC90BAB0B8D0B6E0B4F0B2F0B0F00
:1005C0000AEE0ACD0AAB0A890A650A410A1D09F733
:1005D00009D109A909810957092D090108D308A4DE
:1005E00008740841080C07D5079B075E071D06D84D
:1005F000068E063D05E3057F050B048003C9029DB9
:1000000011C0189589C01895B5C01895A6C048C1EB
:100010001895F1C018951895189518951895189574
:1000200018951895F8948FE592E08DBF9EBFA8951E
:1000300088E181BD8EE181BDA89581E086B98FEF11
:1000400087B98FEF8ABB8BBB80E087BB83E088BB1F
:10005000882784BB8FEF85BB84E881BB88EB82BB9C
:1000600098ED8FEE992EA82E98E0B0E0A0E68827B4
:100070008D939A95E9F785E083BF88278FBD82E04D
:100080008EBD80E0826089BF85B788608B7F85BF29
:100090008BB780688BBF8AB7806480688ABF82E52F
:1000A00088B933B23094442411270027112488E002
:1000B0008093700089E1682EE199FECF82E08EBBCB
:1000C000E09A8DB280927200299912C093B389167A
:1000D00079F090937200892EE199FECF88278FBB2B
:1000E00082E08EBB9DBBE29AE19AA895299BFDCF49
:1000F000BB24CC242227B0E0A0E681E089B980E0CF
:1001000080BD86E880BD8CB188278BB9579A549AF8
:1001100097987894A895FFCF2FB68F939F939DBC07
:10012000ACBC046088B78064806888BF89B780648D
:10013000806889BF8BB78F778BBF3FEFF5E0EEEF1D
:10014000C895902D3196C895802D8A0D991D9BBD1F
:100150008ABD9F918F912FBE18952FB68F939F9335
:100160009DBCACBC89B780648F7789BF8AB7806833
:100170008ABFE3CF2FB68F939F9388E07724F0E078
:10018000E0E6919188949317711C8A9511F0771C81
:10019000F8CF07FF02C0772470947BBA3A953430C9
:1001A000C1F0F4E0E0E08894E30FE30FF11DC8959F
:1001B000902D3196C895802D8A0D991D03975CB5B9
:1001C0006DB5851796070CF4E9CF03969BBD8ABDE4
:1001D0000EC089B78F7B89BF8FEF8BBB89B787FD37
:1001E00006C08AB780688ABF8BB780688BBF9F9133
:1001F0008F912FBE18952FB68F939F939BB18CB183
:1002000093FD25C094FD28C0B39409F4C394213014
:1002100029F0223031F1233058F538C08030B9F45C
:1002200023950260CC24BB24B0E0A0E633B2309426
:1002300044242A9B439488943114410409F026C035
:1002400098E088278D939A95E9F722271FC02227E7
:100250009AE5592E5B981AC021E0809072005C9854
:1002600015C08894B314C40411F42395D4CF0EC0E0
:100270009D9180FE0FD0891719F0AA958D93126079
:10028000879423952C3010F0222708609F918F913E
:100290002FBE18958F3710F4882701C08FEF08956F
:1002A000A8952FB68F936A9431F582E0682E11FDE0
:1002B00025C0389A809170008A958894579450FC94
:1002C00002C0979A01C09798811519F08093700029
:1002D00012C088E080937000882703FF8AE001FF46
:1002E00082E002FF8AEA459902C00F7702C08FEFD1
:1002F0000068582E017F8F912FBE18951D7F389B67
:0C03000002C03898D7CF389AD5CFFFCF75
:00000001FF
